:020000022000DC
:1060000000000120756302005D6302005F6302000F
:106010006163020063630200656302000000000028
:1060200000000000000000000000000067630200A4
:1060300069630200000000006B6302006D630200F0
:10604000A58402006F630200798602006F6302007C
:106050006F6302006F6302002D8502006F63020010
:106060006F6302006F6302006F6302006F630200E0
:106070006F6302006F6302006F6302006F630200D0
:106080006F630200D17502006F6302006F6302004C
:106090006F6302006F6302000DB002006F630200C5
:1060A0006F6302006F6302006F6302006F630200A0
:1060B0006F6302006F630200000000000000000038
:1060C0006F6302006F6302006F6302006F63020080
:1060D0006F6302006F6302006F6302000000000044
:1060E00000000000000000000000000000000000B0
:1060F00000000000000000000000000000000000A0
:10610000000000000000000000000000000000008F
:10611000000000000000000000000000000000007F
:10612000000000000000000000000000000000006F
:10613000000000000000000000000000000000005F
:10614000000000000000000000000000000000004F
:10615000000000000000000000000000000000003F
:10616000000000000000000000000000000000002F
:10617000000000000000000000000000000000001F
:10618000000000000000000000000000000000000F
:1061900000000000000000000000000000000000FF
:1061A00000000000000000000000000000000000EF
:1061B00000000000000000000000000000000000DF
:1061C00000000000000000000000000000000000CF
:1061D00000000000000000000000000000000000BF
:1061E00000000000000000000000000000000000AF
:1061F000000000000000000000000000000000009F
:10620000354936480A1A02D0072291438D4634494F
:1062100034480A1A06D00722914381F309880222E2
:1062200082F3148830483149314A00F044F831484B
:106230003149324A00F03FF831483249324A00F0E1
:106240003AF832483249334A00F035F83248334997
:10625000334A00F030F833483349344A00F02BF821
:1062600033483449344A00F026F83448344900228F
:1062700000F02CF833483449002200F027F8334866
:106280003349091A082902DB002202604160314AC1
:1062900090471F481F49884205D00268043003B464
:1062A000904703BCF7E700208646EC46002000211B
:1062B000294A9047FEE7884207D0521A05D0037852
:1062C00001300B700131013AF9D17047884202D098
:1062D00002700130FAE770470000012000E0002062
:1062E000000001200000012070C50200D82A002013
:1062F000402B0020D0630200D0630200FEB50200F4
:1063000070C50200D82A0020D82A002004B7020055
:1063100004B7020004B7020004B7020004B7020089
:1063200004B7020004B7020004B702006EC5020001
:10633000D8C50200402B0020402B0020402B00201D
:10634000D83D0020D83D0020D83D0020D83D002079
:10635000D85D00209D630200B5960200FEE7FEE7CF
:10636000FEE7FEE7FEE7FEE7FEE7FEE7FEE7FEE705
:1063700000F002B8FFF7FCBF0F484FF00701884359
:1063800085460E4880470E48016841F4700101605F
:10639000BFF34F8FBFF36F8FFFF732BF09480A4932
:1063A0000A4A884207D0521A05D0037801300B7090
:1063B0000131013AF9D1704700000120D57E020079
:1063C00088ED00E004B70200D82A0020D82A002077
:1063D0007047000007B5044B0093044A402300F0C7
:1063E00032F803B05DF804FBF1630200412B00209A
:1063F0002DE9F84388461446B2B10F4B0F4E0325E2
:10640000002743F00109224608EB0701002003F0B2
:10641000EDFA0744241A48B933782BB14FF47A4087
:10642000C847013D02D13570BDE8F88301233370C0
:10643000002CE8D1F8E700BF10B70200402B002085
:10644000704703F003BBF0B595B01D4616460846ED
:106450000C4601F06BFC1A9B0D93CDE908650025F5
:106460002B46082205A920460A958DF82C500C953C
:1064700001F078FC079B0293069B03939DF8143070
:106480008DF8115003F00302012A1DD1BDF814202C
:10649000059DC3F3C203C2F383168DF81030B2001A
:1064A00008230EA9204601F05DFCC5F3952508AB35
:1064B0000093324602AB0EA9284600F02FFB20467F
:1064C00001F038FC15B0F0BD022AF8D1BDF8165025
:1064D000C3F3C203C5F389158DF810300827082DC2
:1064E0002E4628BF08263B4632460EA9204601F01C
:1064F00039FCAD1B08AB02AA31460EA8374400F0A8
:1065000071FB002DEBD1DAE708B5FFF79AFF0448DD
:10651000042100F06DFA034B01225A7108BD00BF3F
:10652000F4B60200D82A0020037813F0040216D033
:1065300003F00303012B03D0022B09D00120704785
:106540000A6800880232C0F3831002440A60F5E74B
:106550000B684288023303EB92130B60EEE71046A0
:10656000704700002DE9F04FDFF81CA187B00F46FF
:1065700000230446861C0DF1070015468DF80730F0
:1065800000F0B8FEDAF804203A60DAF8083003F5D3
:1065900080739B1A0AF21C470AF583690AF21448B1
:1065A000B3421AD30020002D69D004F00F039B01E1
:1065B00043F0050363F30F00DAF80430DAB2033274
:1065C00033444AF822009DF80700CAF8043000F06E
:1065D000B5FE012007B0BDE8F08F0121384601F07B
:1065E000D4F8484601F0E9F8404601F0E6F8DAF858
:1065F00008000290C0B203300AEB800002A9FFF746
:1066000093FF029B30BBDAB20AEB8202D16803919E
:106610009A1C0133DBB20AEB83030292D3F80CB06D
:1066200001F00303012B22D0022B15D083464046F4
:1066300001F0C6F810B1029BCAF808305946384636
:1066400001F0A3F8DAF80830DAF8042003F58073D3
:106650009B1AA5E7D8B2CEE7BDF80E30C3F3891375
:1066600003334FEA1B4B02EB93030293DFE7BDF8C2
:106670000C30C3F383134FEA1B4B1344F5E7A40517
:1066800044F0060098E700BF542C0020064B074852
:1066900010B500221A7001F002FB044610B904483C
:1066A00001F080FB204610BD542C002060B6020093
:1066B0004CB7020030B50A4C71B10A4A0A49121BA4
:1066C000D20800239A4201D1002030BD31F8235076
:1066D000854202D00133F5E7034654F83300F4E76E
:1066E00074B60200F4B60200D82A0020094B013922
:1066F00003EBC000032909D8DFE801F00A02040611
:106700000420704700797047407970470020704737
:106710000220704774B60200034BD3E90130C31A5C
:1067200058425841704700BF542C00202DE9F041D9
:1067300086B0FFF7F1FF0546002840F0ED80774C6A
:10674000C4F81804BFF34F8FA3680293DBB203337E
:1067500004EB830002A9FFF7E7FE029B18B1D4F80F
:106760001824002A5AD0DAB2991C013304EB8202B1
:10677000DBB204EB8303D268DB68049302F003030B
:10678000022B0392029154D1BDF80E306448C3F33A
:106790008917502F3E4628BF502606F1080166F3A0
:1067A0008F13C1F30901ADF80E3001F090FA0546E0
:1067B000002800F09C8001F0B9FA0023082203A908
:1067C000284601F0C5FA0299CB43DBB20133C9B2C6
:1067D0000331B6EB830F4FEA830204EB810125D925
:1067E0005FFA82F80823A6EB0806284601F0B0FA03
:1067F000F6B208F108034B4903F0FC033246284681
:1068000001F0A6FA029B033703EB97070297D4F82F
:106810001834002B43D1D4F8106453E062689A42D4
:1068200094D8A260284606B0BDE8F081082332461D
:10683000E5E7012B5BD1BDF80C303948C3F3831178
:10684000062928BF062161F38913023101F00F01E7
:106850008900ADF80C3001F03AFA0546002846D020
:1068600001F064FA0023082203A9284601F070FA17
:106870000026BDF80C20C2F38312B300964203F148
:106880000803C4D202994A1CC9B20331029204EB34
:1068900081010422284601F05BFA0136E9E7284627
:1068A00001F048FAFFF738FF80F00100C5B2B9E700
:1068B000F3685B7923B1336829461B6830469847F3
:1068C000F3681E68002EF3D1284601F033FA0DF16B
:1068D00007008DF8076000F00DFDD4F818340BB9EF
:1068E000029BA3609DF8070000F028FDDAE7D4F8CA
:1068F000104454B90C4B0D480D49C01AC00800048F
:1069000040F0020000F05CF8CCE7236820469B686A
:106910009847E3681C68ECE7002583E7542C0020C7
:1069200060B60200602C002074B602009CB6020023
:1069300034B702002DE9F34704460E46924601A9FA
:10694000012218469946FFF70DFE1B4F10B3019D1B
:106950004FF00008AA1CC84508EB020123D11748D4
:10696000002100F0E3FE80F31000000440EA144030
:10697000E4006B1C04F03804DBB2EDB244F0010417
:1069800007EB8303033544EA881444EA8624D8607D
:1069900047F825403B781BB1FFF7C8FE0028FBD124
:1069A00002B0BDE8F087C9B207EB81015AF8283080
:1069B000CB6008F10108CEE7542C00207030002095
:1069C00000231A46FFF7B6BF07B50123019201AABB
:1069D000FFF7B0FF03B05DF804FB07B5CDE9002376
:1069E00002236A46FFF7A6FF03B05DF804FB000030
:1069F00030B50F4CD4F8102403460020114631B9AD
:106A0000D96808714AB9C4F810340A6030BDC96841
:106A10000D79854206D00968F1E7D26814680C60E8
:106A20001360F3E701300A28E8D14FF0FF30EDE7BB
:106A3000542C002038B5084B0125D3F810441D70A4
:106A400004B938BDE3685D71236820465B689847E8
:106A5000E3681C68F4E700BF542C002030B5C388FD
:106A600085B004460D4633B1144A00921449154AC4
:106A7000284600F008FF217A05291DD0637A4BB122
:106A8000A088FFF733FE104B104953F8202028460A
:106A900000F0F9FE227A0E4BA08853F822200392D0
:106AA0000021FFF707FE039A0A490346284605B06E
:106AB000BDE8304000F0E7BE05B030BD78B7020059
:106AC00060B7020058B70200E4B702007DB70200C9
:106AD00008B8020080B7020007B503460846197AD5
:106AE000052911D05B7A2BB1094A0A49019000F0BF
:106AF000CAFE01980849019000F0C5FE019803B054
:106B00005DF804EB00F0B4BE002AF8D0F2E700BF55
:106B100078B702007DB7020075B702002DE9F04397
:106B200085B01F460C9D002395F80C902B730646EC
:106B30000C46904629463846FFF790FFB8F1060FFD
:106B400009D8DFE808F00412181F28334000314646
:106B5000284600F098FE002229463846FFF7BCFF81
:106B600085F80C9005B0BDE8F083226831462846D0
:106B700000F089FEEFE7D4E900233146284600F013
:106B800082FEE8E7A36800933146D4E90023284653
:106B900000F079FEDFE7E3680193A36800933146D4
:106BA000D4E90023284600F06EFED4E7236902935F
:106BB000E3680193A36800933146D4E90023284693
:106BC00000F061FEC7E76369039323690293E368FA
:106BD0000193A36800933146D4E90023284600F0CE
:106BE00052FEB8E708292DE9F74F80460E461746B2
:106BF0001C463DD800251B7B25732146104601937A
:106C0000FFF72CFFDFF88CA0DFF88CB0AE4232D952
:106C100018F805205946204600F035FE0135082DAC
:106C2000F4D11B49DFF874A0DFF874B0204600F0FF
:106C30002AFE4FF000094E4524D918F809507E2D40
:106C40001ED8284604F00AFC002814BF2A462E222B
:106C50005946204600F017FE09F10109B9F1080F65
:106C6000E9D1012221463846FFF736FF019B237305
:106C700003B0BDE8F08F5146204600F004FECDE79A
:106C80002E22E5E75146204600F0FDFDE4E700BF77
:106C900094B7020090B702008AB7020092B70200D0
:106CA00096B702001FB50021039001AA44F201002B
:106CB000CDE9011100F004F805B05DF804FB000017
:106CC00038B572B6FFF7B6FEFFF730FD0028FBD1EE
:106CD000104B114C114D1249E41AE408240444F0FD
:106CE0000100FFF76DFED5F8F030DB0700D500BEE0
:106CF0000C4944F00200FFF763FEBFF34F8FEA68D0
:106D0000094B02F4E0621343EB60BFF34F8F00BF07
:106D1000FDE700BF74B602009CB6020000ED00E083
:106D200027B8020033B802000400FA0549B152B195
:106D3000531E1A4007D1826001608380C2601046F2
:106D400070470E2070470920704710B58468C268EC
:106D50008388121B934208D3C26813400268D1543F
:106D6000C3680133C360002010BD0420FCE78268C3
:106D7000C3689A420AD08268838813400268D35C51
:106D80000B708368013383600020704705207047D3
:106D900010B5D0E90243D1E90202A04272EB03032D
:106DA0002CBF0120002010BD08B50A4800F0F9FBF7
:106DB000094AD2E90031C018084BD3E9002341F158
:106DC0000001904271EB030303D210F1807041F196
:106DD000000108BDE02A0020103100208831002089
:106DE00037B505460C460A4801A900F00EFC60B113
:106DF0000570446001A9064800F031FC18B105484F
:106E000000F0D4FB002003B030BD0420FBE700BF3E
:106E100074310020E02A002038B5184B1B78044656
:106E200013B90025284638BD0028FAD0037F03F0A7
:106E3000FF05002BF5D0FFF7B7FFD4E902239042FE
:106E400071EB030314D3236903B92377D4E9053025
:106E5000984721690029E4D0237F03F0FF05002B28
:106E6000DFD0D4E902325B1842F10002C4E90232F9
:106E70000348214600F0B5FFD4E700BF18310020D9
:106E800050B8020013B5114B11491868019008233E
:106E90001048582200F0A6FB044698B90E4A0F4845
:106EA00001A900F06FFA044660B90C48012100F016
:106EB0005BFB01230A4A0948194600F0BDFA094B59
:106EC00001221A70204602B010BD00BF4AB802006D
:106ED0001C31002074310020496F0200E02A00209C
:106EE000FFFF7F00183100203AB103685A614A1E43
:106EF000514251411961002070470720704738B551
:106F0000037F04460D4683B98261FFF74DFF236975
:106F1000281841F10001C4E9020103B125612146AD
:106F20000020BDE83840FFF75BBF002038BD0023DC
:106F3000014603770120FFF753BF0000014800F02E
:106F400030BB00BFE02A00202DE9F347064600F0E1
:106F500013FB40B1584AD2E9003113F1807341F17B
:106F60000001C2E900310021304600F014FB38B1C5
:106F7000524C236823B12068FFF74EFF00232360A3
:106F80000121304600F007FB20B1FFF70DFF4C4B0D
:106F9000C3E900014B48494D4B4C4C4F01A900F04F
:106FA0006EFB002842D1DFF82081444CDFF82491A9
:106FB000404600F02CFF2368002872D07BB1236884
:106FC000D0E90252D3E902138D4272EB03032AD2B5
:106FD00023681B7F1BB12168404600F002FF40463A
:106FE00000F00FFFD0E9027A0546FFF7DDFE381A00
:106FF0006AEB010A01287AF1000345DBB0F5350F91
:1070000040D3FFF79BFF324A02444FF4960300211E
:10701000484600F031FA00283ED1236813B93046C3
:1070200000F002FA256002B0BDE8F0870378012B7A
:107030001DD0022B09D14FF00008204600F0E1FEE0
:10704000002836D080F81C80F7E73BB941680B7FF9
:1070500023B901230B77204600F0C3FE01A919488C
:1070600000F038FB01A9174800F009FB99E74168D7
:107070002B68994202D100232B60EFE7204600F0F5
:10708000C9FEEBE7AA68C0E70021484600F079FA9C
:107090002846FFF7C1FE01E00D28F9D00023236048
:1070A00086E7002BBFD1304602B0BDE8F04700F0C4
:1070B000BFB901233B70D1E710310020903100208F
:1070C000883100207431002050B8020018310020AF
:1070D000FFFFB400E02A00200648074A037807496A
:1070E000D35C012213B1043001F026BF0C3001F053
:1070F000E9BC00BFE82A002004320020BC31002097
:107100000648074A03780749D35C012213B10430CB
:1071100001F0C4BE0C3001F085BC00BFE82A00209D
:1071200004320020BD31002037B50578012D0DD087
:10713000022D30D075B91F491F48FFF718FE0028EF
:1071400034D103B0BDE83040FFF7DABF037A1BB992
:10715000FFF7C2FF03B030BD4368184C19782046D2
:10716000FFF7F3FD80B18DF800500190144B684695
:107170001B689847A168E368A2885B1A9A42E7D225
:10718000104B01221A70E5E7A268E3689A42F1D039
:107190008DF80000EAE7C3688DF800500193FFF70F
:1071A0009BFF074B68461B689847D3E703238DF87E
:1071B0000030F6E7BD310020AC31002098310020CE
:1071C00094310020A8310020F0B51F46234B89B030
:1071D00004461A600D4600293DD08A882048096877
:1071E000FFF7A4FD002834D1AA89A9681D48FFF73C
:1071F0009DFD00282DD11C4E0FCE6D460FC596E883
:107200000F0085E80F0063690693237C174A18482E
:107210008DF81C70003B18BF01238DF81430637C7F
:10722000002B14BF0E2300238DF81530E368029362
:10723000A36803932368019369466368009301F090
:10724000B9F830B90B4B18702368013301D0FFF740
:1072500043FF09B0F0BD0720FBE700BF94310020D9
:1072600098310020AC3100205CB802002971020086
:10727000E82A0020A831002070B5084D01460848D2
:107280002E78FFF774FD044636B100232B70FFF70C
:1072900023FF08B1FFF706FD204670BDA83100208E
:1072A0009831002010B501460E48FFF74EFD044608
:1072B000A8B90D480D4A0378D35C63B1043001F0DE
:1072C000E1FD60B90A490748FFF751FD38B9BDE84B
:1072D0001040FFF715BF0C3001F098FBF1E7204696
:1072E00010BD00BFAC310020E82A0020043200208D
:1072F000BD31002070B5EFF3108672B60C4A946869
:1073000001239CB993600B4B0B4DD3F8801029409F
:107310001160C3F88050D3F8841051604FF0FF32F1
:10732000C3F88420047006B962B670BD0370FAE732
:10733000C031002000E100E0FC06FFBD084B9A6868
:1073400010B55AB150B9EFF3108172B6054A1C68F6
:1073500014605C685460986001B962B610BD00BFEB
:10736000C031002000E100E0435882B03BB100236F
:10737000435043580193019B012002B070471846C7
:10738000FBE70000F8B5204B4479204E43F8242059
:107390001F4A204B06EBC4049B1A2279DB081B040E
:1073A00032B143F002001C49FFF70AFB0820F8BD88
:1073B00002680C88C2F8084590F904508A7804796C
:1073C0005201002DD2B219DB14494F1987F800235E
:1073D00001226D0904F01F0402FA04F441F825406B
:1073E000427906EBC201012446F832000C7143F0E9
:1073F00003000B49FFF7E4FA0020D8E7094904F03D
:107400000F040A55ECE700BFD4310020CC31002036
:1074100074B60200ACB602007CB8020000E100E0E5
:107420009EB8020014ED00E0036801221A60704764
:10743000036801225A60704773B501F15005AD0031
:107440000068ADB24FF480348C400026C0F8084389
:10745000C0F84843465101F5A8714559019522F0FD
:107460007F42019D40F82120C0F844430BB1C0F891
:10747000044302B070BD00002DE9F74F0D4622F025
:107480007F4402684FF4803705F150068F408046F4
:10749000B60002EB8500C2F84873B6B2C2F80873B2
:1074A000D2F8041599464FF0000BD0F84035C0F8DB
:1074B000401542F806B05B1A9259009223F07F43C0
:1074C000012B009A4FEA850A0CD1264B4FF48060BD
:1074D00043F001039847D8F8003043F806B09B59B1
:1074E0000193019BD8F80010D1F80465C1F84473EA
:1074F000A31B23F07F43012B1CD11A4B05F5A87564
:10750000013443F0010341F825404FF4806098476F
:10751000D8F80030D3F804359E4209D1D8F80030AD
:107520000020C3F84473C3F8047303B0BDE8F08FC0
:107530000D20FAE78A44C9F1FF13CAF84045D1F893
:107540000405221A013A22F07F4203F57F43934259
:10755000EED3002AE2D10134CAF84045D1F804350F
:107560009842DAE7B0B8020003680222C3F8442365
:1075700009B1C3F80423704700684FF48271FFF724
:10758000F3BE4FF4803303FA01F10368C3F84813E4
:10759000C3F80813704750318900006889B2FFF7BB
:1075A000E3BE0368D3F804057047000090F9043087
:1075B000002B09DB5A09012103F01F0301FA03F331
:1075C0004032024941F82230704700BF00E100E03C
:1075D000024B034A1B681068184700BFD4310020D3
:1075E000CC31002010B561B1B2FBF3F403FB1424DD
:1075F000A4B244B9C0E9001484608281C3812046EA
:1076000010BD0E20FCE70920FAE737B550E8013F2E
:107610009DB2C48925448489A54228BF2D1B0489B5
:10762000A54202BFBFF32F8F002207E0C5EA030582
:1076300040E80154002CE9D14FF001028DF80320FD
:107640000193019A0A609DF8031001F0FF0321B134
:10765000006810FA82F003B030BD1846FBE70A88D4
:107660004B889A4209D150E8012FC2EA024240E811
:107670000123002BF7D1012070470020704737B558
:1076800050E8023F1FFAA3F5C488A54202BFBFF32A
:107690002F8F00220DE0C48925448489A54228BF8C
:1076A0002D1BC3EA054540E80254002CE8D14FF0F9
:1076B00001028DF803200193019A0A609DF80310DE
:1076C00001F0FF0321B1006800EB124003B030BDB0
:1076D0001846FBE70A884B889A4209D150E8022FE6
:1076E000C2EA224240E80223002BF7D10120704772
:1076F0000020704701F01F024B090121914000EB6F
:10770000830000F01EB801F01F0301229A404B09CC
:1077100000EB8300D14300F02CB84B0901F01F01AE
:1077200050F82300C84000F00100704710B5034630
:1077300053E8000F0A4643E8002494F0000FF7D105
:1077400010BD10B5034653E8002F42EA010043E89C
:10775000000494F0000FF6D110BD10B5034653E8B5
:10776000000F00EA010243E8002494F0000FF6D174
:1077700010BD10B5034653E8002F02EA010043E8AC
:10778000000494F0000FF6D110BD10B5034653E885
:10779000002F02EB010043E8000494F0000FF6D143
:1077A00010BD10B5034653E8002FA2EB010043E8DB
:1077B000000494F0000FF6D110BD0121FFF7C1BF06
:1077C0000021FFF7CABF10B590B1D0E901230168CD
:1077D0009B1ADBB20A60013BDBB2FF2B026802D1CD
:1077E0000020107110BD11684C1C14600B70F2E782
:1077F0000E20F7E737B5054600240DF107008DF898
:107800000740FFF777FD2A686B68116899420ED927
:10781000481E106011F8013CEC68298A01FB034402
:10782000AB6811791B1ADBB2994238BF13719DF80E
:107830000700FFF783FD204603B030BD37B505468E
:1078400000230DF107000C468DF80730FFF752FDBD
:107850002A681368591C1160E968641A298AB4FB04
:10786000F1F41C709DF80700FFF768FD03B030BD10
:10787000826810B504462AB14369016800699847D7
:107880000023A36010BD0EB403B5039921B104AB6E
:1078900001AA019300F076F802B05DF804EB03B0A2
:1078A00070470A2938B504460D4602D10D21FFF76D
:1078B000F8FFA3682268591CA160D554D4E90132AD
:1078C0009A4204D32046BDE83840FFF7D1BF38BD07
:1078D0002DE9F84F9846DDE90A43154682460F46E2
:1078E0000A464FF00109AA420FD2C14538BFC1462E
:1078F00013F0010B01D16CB900240126B8F1010F7E
:107900001BD908F1FF386E43F8E709F10109B2FB12
:10791000F5F2E8E79B070ED5B8F1000F0CBF302653
:107920002026A145E9D2013C31465046FFF7B9FF78
:10793000002CF6D1E0E72026F3E7B7FBF6F39D42F3
:10794000E1D9DFF83C80B7FBF6F3504618F8031096
:1079500006FB1377FFF7A5FF3346AB42B6FBF5F600
:10796000F1D2BBF1000F02D00CB1A14501D3BDE8AB
:10797000F88F20215046013CFFF793FFF4E700BF4A
:10798000B6B802002DE9F74F05461746884600298C
:1079900000F03E8118F8011B49B92B7B002B00F049
:1079A0003781284603B0BDE8F04FFFF761BF2529B6
:1079B00040F0B780002698F800302D2B424608F1A1
:1079C000010823D0302B24D02B2B25D000242A2BA8
:1079D00002F1010123D13B681A1D1B683A601C4467
:1079E0000A4613782E2B26D101324FF0000A10469A
:1079F00010F8011BA1F1300CBCF1090F1DD80A23AE
:107A000003FB0A13A3F1300A0246F0E746F0010631
:107A1000D1E746F00206CEE746F00406CBE711F8C0
:107A2000013CA3F130000928DBD80A2202FB043410
:107A3000303C0A46CBE74FF0000A12F8011B01F078
:107A4000FB0068289046F8D0782909D86F290CD80F
:107A5000632962D022D8252963D0582900F0888074
:107A600098F80030002B95D197E770390829F7D89E
:107A700001A353F821F000BFEB7B0200617A020002
:107A8000617A0200817B0200617A02005F7B020062
:107A9000617A0200617A0200717B0200642901D0E0
:107AA0006929DDD13A68D2F80090111D89EAE9729E
:107AB0003960A2EBE9724FF0010B092A35DCD3459E
:107AC00038BFD3462CB1B9F1000F01DB720700D5E6
:107AD000013CB30702D5BAF1000F03D0F00701D47F
:107AE0004CBB0024B9F1000F2DDAC9F100092D219A
:107AF0002846FFF7D6FE06F00302022A04D1BAF1A7
:107B0000000F01D11CBB0024CDE9004653460A22D8
:107B100049462846FFF7DCFEA2E73B681A1D1978A4
:107B20003A602846FFF7BDFE9AE70A230BF1010BE6
:107B3000B2FBF3F2C1E7A345D4D220212846013C91
:107B4000FFF7AFFECCE77107D5D52B21D0E7A345D2
:107B5000DAD230212846013CFFF7A3FED2E739688C
:107B6000CDE900460A1D3A6053460A220968D0E76B
:107B700039680A1D3A60CDE9004653461022F5E700
:107B80003B681A1D3A6016F00106D3F8009024D124
:107B9000B9F1000F03D0484603F0FFFC0646B4429B
:107BA0001DD809F1FF3919F8011F00293FF458AF1A
:107BB0002846FFF776FEF6E728460136FFF771FE06
:107BC00019F806100029F7D1A642BFF449AF2021C9
:107BD0002846013CFFF765FEF6E70026F0E7202186
:107BE0002846013CFFF75DFED9E73B681A1D3A6065
:107BF000302128461C68FFF754FE78212846FFF7FD
:107C000050FE00220823CDE900322146102280E7F1
:107C100003B0BDE8F08F00BF2DE9F84FB0F806A023
:107C20004579D2F800B09DF828900AFB05F5043D8F
:107C300088460BEB0301A94203F1040488BFA5EBBE
:107C4000030BB4FBFAF607460AFB1644C2F800B071
:107C50004EB9AAEB04055D4528BF5D46BBF1000F98
:107C600004D1BDE8F88F3F68013EF1E7043408EB2A
:107C700006003C442A46B9F1000F0DD02146ABEB7B
:107C8000050B03F00CFCDA452E443F6855464FF0D7
:107C9000000428BF5D46E1E701462046EFE7FFF715
:107CA00092BDF8B546790146721E054600239342FF
:107CB0002D6803D30024A64202D8F8BD0133F6E7AD
:107CC0000F682846FFF7BAFD01343946F3E72DE97E
:107CD000F843068ACD1C0746FFF78CFD043E354469
:107CE0000446B5FBF6F5F0B14FF48073EDB2838036
:107CF000C680013D076081464FF00008A84512D2BA
:107D00003846FFF777FD064648B163790133637162
:107D100008F10108C9F8000007608146EEE7204637
:107D2000FFF7BFFF34462046BDE8F8830121043049
:107D3000FFF72BBD10B5012104460430FFF731FDDC
:107D4000C0B220B92046BDE81040FFF7AABF10BD61
:107D50001FB503920022009203AAFFF75DFF05B052
:107D60005DF804FB1FB503920122009203AAFFF7FE
:107D700053FF05B05DF804FB064B10B500241C70E2
:107D8000054B1C60BFF35F8F0449054800F013F8F2
:107D9000204610BDE0310020E4310020D0B80200C0
:107DA000D8310020836800225A60C3E904229A6017
:107DB000DA601A6070470B684A684360934208BFF4
:107DC0000023016008BF43607047436843B1026805
:107DD000916852680B449342436004BF00234360A0
:107DE000704770B5446806460D46206818B1B36800
:107DF0002946984718B923682B60256070BD246810
:107E0000F3E74368186808B102681A60704743686E
:107E1000186870474368186800B97047884203D1F2
:107E200002681A600120704703460068F4E700000A
:107E300010B50D49A1F59472914201D800200FE0D0
:107E40008C1AE30F03EBE4035B1002EBC30452F85C
:107E50003330834205D802D204F10802ECE76068AF
:107E600010BD2146E8E700BFDCBD020008B5FFF702
:107E7000DFFF024B002808BF184608BD9FBC020068
:107E800010B50446C0B2FFF70DFA204610BD4FF002
:107E90008053D3F83001421C04BF4FF0704393F875
:107EA000E00F831F58425841704700004FF0704365
:107EB00093F8E02F062A09D1D3F8E83FC3F3031360
:107EC000033B032B02D8024AD05C70470020704766
:107ED000E4BD020008B5FFF7DAFF40B14FF0805370
:107EE0008F4AD3F82433C3F30423C2F84035FFF795
:107EF000DDFF10B18B4B8C4A5A67FFF7C8FF48B1C2
:107F00004FF080534FF08042D3F84432C3F34233F2
:107F1000C2F83C35FFF7CAFF30B1844AD2F8FC30D2
:107F200023F08073C2F8FC30FFF7B1FF40B14FF08F
:107F300080430022C3F80C21C3F81021C3F8382570
:107F4000FFF7B4FF20B14FF080430322C3F8A02510
:107F5000FFF7ACFF60B1764B0522C3F81026012273
:107F6000C3F888260022C3F818263F22C3F8142637
:107F70004FF08053D3F83021511C09BF4FF07043AC
:107F8000D3F8343193F8E02FD3F8E83F08BFC3F3B8
:107F90000313062A4DD1033B032B03D8654AD35C58
:107FA000002B46D04FF08052634BD2F80414C3F834
:107FB0002015D2F80814C3F82415D2F80C14C3F80D
:107FC0002815D2F81014C3F82C15D2F81414C3F8DD
:107FD0003015D2F81814C3F83415D2F81C14C3F8AD
:107FE0004015D2F82014C3F84415D2F82414C3F86D
:107FF0004815D2F82814C3F84C15D2F82C14C3F83D
:108000005015D2F83014C3F85415D2F83414C3F80C
:108010006015D2F83814C3F86415D2F83C14C3F8CC
:108020006815D2F84014C3F86C15D2F84424C3F88C
:108030007025FFF72CFF48B14FF080534FF080427E
:10804000D3F8583203F04F03C2F8E43EFFF71FFFA6
:1080500048B14FF08043D3F80024D20744BF6FF0FB
:108060000102C3F800244FF08053D3F83021062AD0
:108070000ED1D3F83431033B032B02D82F4AD35C03
:1080800033B12F4AD2F83C3743F48063C2F83C370F
:10809000264AD2F8883043F47003C2F88830BFF320
:1080A0004F8FBFF36F8F4FF01023D3F80022002AB9
:1080B00003DBD3F80432002B2EDA224B0122C3F863
:1080C0000425D3F80024002AFBD04FF010221521FC
:1080D000C2F80012D3F80024002AFBD04FF010237E
:1080E0001522C3F80422174BD3F80024002AFBD032
:1080F0000022C3F80425D3F80024002AFBD0BFF3E4
:108100004F8F0A49104BCA6802F4E0621343CB60F8
:10811000BFF34F8F00BFFDE70C4B0D4A1A6008BD3F
:108120000030014000C007400DF0ADBA00ED00E0A6
:1081300000500040DCBD020000C00040E0BD020075
:108140000010004000E001400400FA05FC2A002075
:108150000090D003054A4FF0A043105CD3F80435DB
:1081600023FA00F0C04300F001007047ECBD0200AC
:10817000044B1A5C012393404FF0A042C2F80C3527
:10818000704700BFECBD0200044B1A5C0123934012
:108190004FF0A042C2F80835704700BFECBD0200A6
:1081A00008B50020FFF7F0FF0120FFF7EDFF0220E8
:1081B000FFF7EAFFBDE808400320FFF7E5BF08B579
:1081C0000020FFF7D5FF0120FFF7D2FF0220FFF7C5
:1081D000CFFFBDE808400320FFF7CABF074A4FF0B2
:1081E000A041105CD1F804350122824022EA03004C
:1081F0001340C1F80805C1F80C357047ECBD02000A
:10820000014B185C704700BFE8BD020038B5074C51
:10821000051E04F1080318BF1C4623682BB11A6819
:1082200022605B6828469847F7E738BDF0310020A8
:1082300020B9054B01225A70FFF7E8BF012802D18F
:10824000014A9070F8E77047E831002020B9034BED
:1082500001225A70FFF7DABF704700BFE8310020F3
:1082600038B50E4C2378B3B90D486360A360236121
:10827000E36000F0E7F8054602F0AEFE08B900F052
:10828000EDF801232370074BD3F800340BB1012321
:10829000A370284638BD8525F5E700BFE8310020EA
:1082A000318202000000014037B50D4C00230DF172
:1082B00007008DF80730FFF71DF8E368013BE36026
:1082C000E36833B9074BD3F8005415B900F0D8F878
:1082D000A5709DF80700FFF731F803B030BD00BF6F
:1082E000E831002000000140012813B50CD003281C
:1082F00020D038B9134B0122C3F88020BFF34F8F31
:10830000BFF36F8F02B010BD0F4C00230DF10700BB
:108310008DF80730FEF7EEFF23780BB9FFF7A0FFCB
:10832000E3689DF807000133E3600123A370FFF7C2
:1083300005F8E7E700F092F802B0BDE81040FFF75B
:10834000B3BF00BF00E100E0E83100201FB50378B3
:108350008DF800304368019383688DF80830C36856
:10836000054A0393054B684653F8213052F8211013
:10837000984705B05DF804FBFC3100200032002076
:108380001FB503788DF800304368019383688DF83A
:108390000830C368054A0393054B684653F82130FB
:1083A00052F82110984705B05DF804FBFC3100201D
:1083B00000320020F0B5194B90F800C091F81DE094
:1083C00043F82C20164B16460A6943F82C20154B0F
:1083D00003F80CE00C4607460FCC89B06D460FC57C
:1083E00094E80F0085E80F00CDF810C0BEF1000F33
:1083F00009D0002E0C4A694608BF3246381D00F0ED
:108400007FFC09B0F0BD002E084A694608BF32461D
:1084100007F10C0000F046FAF3E700BF003200203D
:10842000FC310020043200204D83020081830200D1
:1084300000F18040002382B0036003680193019B38
:1084400002B07047044A137923B90121106091806A
:10845000184670478520704708320020074B1A687D
:10846000D20704D4C02283F8002301221A604FF0FF
:1084700080430122C3F81825704700BF00E100E0E7
:108480004FF0804208B50223C2F808334FF48270DF
:10849000FFF7CEFF0123D360D2F81834DB03FBD4FF
:1084A00008BD00004FF0804110B5D1F8003163B134
:1084B0004FF48070FFF7BCFF0D4B58790122C1F8D3
:1084C000082310B95A711B6898474FF08042D2F8C0
:1084D000043163B14FF48270FFF7AAFF0223C2F8A0
:1084E0000833034BBDE810401B680120184710BD3E
:1084F0000832002000F1804000F5C040002382B027
:10850000036003680193019B02B07047800000F193
:10851000A040D0F8002722F44032C0F80027D0F85D
:10852000003743EA0141C0F8001770472DE9F74FC3
:1085300000244E4D01944FF48072012102F18043DA
:1085400003F5C04390B21B68012B06D1D5F8043364
:108550000B4202D0FFF7CEFF0C430432B2F5907FFE
:108560004FEA4101EAD1414BD3F87C31012B0CD1C8
:108570004FF4BE70FFF7BEFF4FF0A04344F000443D
:10858000D3F820250192C3F82025E3B2D3B1384FA8
:1085900000250126344210D0AB0003F1804303F5DF
:1085A000C043D3F81005D3F8101557F8253023B180
:1085B000C1F30141C0F3042098470135082D4FEA6B
:1085C0004606E7D1002C48DA294D4FF0A048294E45
:1085D0004FF00009012716F9013B5A1C31D0C3F3B3
:1085E000C20202A90A44DCB212F8042C03F03F0ACA
:1085F00003F0070307FA03F31A4222D00AF5E073E7
:10860000504658F82330C3F3014BBBF1020F0CBFA7
:1086100003210221FFF77AFF07FA0AF3C8F8203591
:1086200005EB0A0393F9303055F823304BB1A1091B
:10863000032904D0BBF1020F12D1012901D1504608
:10864000984709F10109B9F1040FC4D1D8F82035D0
:108650000193C8F82035002BB9D103B0BDE8F08FE5
:10866000BBF1030FEDD10229E8E700BF0060004035
:108670001032002060320020014B1B68184700BFF9
:108680006C3200200E4B984237B50C4602D00020C9
:1086900003B030BD00230DF107008DF80730FEF761
:1086A00029FE084B1D7915B901221C601A719DF82D
:1086B0000700FEF743FE002DE9D01120E8E700BFD8
:1086C000002000406C3200200023435082B0435809
:1086D0000193019B02B070470A4610B54FF48E71AA
:1086E000FFF7F2FF136A9168C95C136A01331362E2
:1086F000C0F81C1510BD024608B500684FF4927111
:10870000FFF7E2FF10684FF48471FFF7DDFF136895
:1087100001221A6008BD8B690A4610B54FF48471B6
:1087200023B9FFF7D1FFD0F8183510BDFFF7CCFF04
:10873000536AD168D0F81805C854536A013353629C
:10874000F3E700001FB501238DF80030044BCDE99D
:108750000110D3E900126846904705B05DF804FBAC
:108760007432002030B54D4DD5F804339A0585B0EC
:1087700051D5D5F82431002B4DD04FF492712846B5
:10878000FFF7A2FF4FF40173C5F80833444B93F889
:1087900029200AB901226A60404902228DF800208E
:1087A000D1F88024C1F8802403929A690292DA6891
:1087B00001920022C3E906226846D3E900129047DD
:1087C0003648D0F81C315BB1354A5169136A994279
:1087D0004DD992F82830002B49D11146FFF77CFF84
:1087E0002E48D0F84431002B56D04FF4A271FFF739
:1087F0006BFF2B4B93F829200AB1012202609A6982
:10880000002A49D0586AD96800229A6105B0BDE8AB
:108810003040FFF797BFD5F804335B07D0D5D5F8C4
:108820000831002BCCD01E4C1C482146FFF773FFAB
:10883000636AA2699A42C3D1E369E1684BB1A3615B
:108840002369E3600023606AE3616362FFF77AFFF4
:10885000B6E794F829300BB901236B600F4B4FF446
:108860000172C3F808230023606AA361EEE70B4896
:108870004FF48E71FFF728FF5369002BB0D0516978
:108880000291002391688DF8003001915361684690
:10889000D2E900139847A3E705B030BD002000409F
:1088A000743200202DE9F843534D90F804802C23B6
:1088B00003FB0853064693F82A300C469146002BDA
:1088C00040F096804D490068FFF7DCFE074600281F
:1088D00040F0908022683068511C0BD04FF0A041CE
:1088E00001239340C1F8083502F5E0734FF0030C03
:1088F00041F823C061684B1C1FBF01F5E0734FF0C6
:10890000A04C4FF0000E4CF823E0A369C0F82435CA
:1089100094F814C0637DBCF1010F4CEA0303C0F866
:108920006C35C0F81415C0F80C251DD1A268531C75
:108930001FBF02F5E0734FF0A0414FF0000C41F86B
:1089400023C0E368591C0BD04FF0A04C0121994083
:10895000CCF8081503F5E0714FF0030E4CF821E058
:10896000C0F80835C0F810252C2202FB08F2AB181D
:10897000C3F804902369AB50B9F1000F20D04FF435
:108980008E71247FFFF7A0FE4FF4A2713068FFF7CD
:108990009BFE32681A4BC2F80433130B42F30732C2
:1089A0006101002AC9B21EDB1648841884F800133E
:1089B0000121520903F01F0301FA03F340F82230AA
:1089C00033680422C3F800252C2303FB085300223C
:1089D000C3E9062283F829205A61012283F82A205C
:1089E0003846BDE8F883084A03F00F03D154E7E79F
:1089F0000827F5E71127F3E77432002065870200A6
:108A00008000020000E100E014ED00E00279044B78
:108A10002C2101FB02335869003818BF0120704730
:108A2000743200202DE9F84F064690F804808946FC
:108A30009246FFF7EBFF044600283CD1204F2C253F
:108A400008FB057B4FF48E71CBF814A0CBF808908F
:108A5000CBF820008BF828003068FFF735FE30682F
:108A6000012383605946FFF737FEDBF804305D468B
:108A70001BBB3068DBF814402B6A9C4211D833686A
:108A8000D3F81C21002AFBD00122DA6000202C231D
:108A900003FB087700237B61BDE8F88F95F8283049
:108AA0003BB9D0F81C31002BF8D05946FFF714FE23
:108AB000E2E70F20EBE71120EEE72046ECE700BFEE
:108AC000743200202DE9F0473A4D07792C2303FB3F
:108AD000075306465C6824B103684FF40170C3F87D
:108AE00008032C2303FB0753986950B1D869002869
:108AF00041D024B133684FF40172C3F80423112428
:108B000036E09A61D9605862D8612C2303FB075381
:108B100093F829301BB910B93046FFF7ECFD4FF040
:108B20002C0808FB075A3068DAF80430002B37D1DC
:108B30004FF4A271D046FFF7C7FD3068D0F82491FA
:108B4000D0F80831D0F84441CBB914B9B9F1000FCD
:108B5000F3D02C2303FB07550023AB61B9F1000FC1
:108B600024D12CBB95F8291033680122B1B11A60C9
:108B70002046BDE8F0871961DA610120C5E7B9F147
:108B8000000FE6D1002CE4D14146FFF7C4FDDAF82E
:108B90002430DAF818209A42CFD8DAE75A60E7E7AB
:108BA0004FF40173C0F804330024E1E70324DFE746
:108BB0000F24DDE7743200200023435082B0435875
:108BC0000193019B02B070471FB501238DF800305F
:108BD000044BCDE90110D3E900126846904705B077
:108BE0005DF804FBA03200207FB5434AD2F824612F
:108BF000002E60D010464FF49271FFF7DDFF022384
:108C00008DF80030D2F88034C2F880340393D2F863
:108C10003C350293394BDA6801920022C3E90622FF
:108C20006846D3E9001290473348D0F8443173B115
:108C30004FF4A271FFF7C0FF304B9A693AB100229E
:108C4000C3E90622D968D0F83C05FFF7BDFF2A48E2
:108C5000D0F82031ABB14FF49071FFF7ADFF012395
:108C6000C360264B5A6962B1D0F84C1502910022BC
:108C700099688DF8002001915A616846D3E9001285
:108C800090471D48D0F858319BB14FF4AC71FFF7B5
:108C900093FF1A4B5A6962B1D0F84C150291002229
:108CA00099688DF8002001915A616846D3E9001255
:108CB000904704B070BDD2F81031002BB4D04FF4FF
:108CC00088711046FFF778FF0C4BD2F83C05996984
:108CD0008842A9D1DC69D96864B1D2F8005225F084
:108CE0002005C2F800521A699C61DA60DE61FFF764
:108CF0006BFF99E79C61FAE700200040A03200205A
:108D00002DE9F8435A4E90F80480242303FB0863AE
:108D1000044693F820300D469146002B40F0A38086
:108D200054490068FFF7AEFC0746002840F09D80DC
:108D30002A682068511C0BD04FF0A04101239340BA
:108D4000C1F8083502F5E0734FF0030C41F823C079
:108D500069684B1C1FBF01F5E0734FF0A04C4FF04A
:108D6000000E4CF823E0AB69C0F8243595F814C028
:108D70006B7DBCF1010F4CEA0303C0F86C35C0F801
:108D80000C25C0F814151DD1AA68531C1FBF02F58D
:108D9000E0734FF0A0414FF0000C41F823C0EB68A6
:108DA000591C0BD04FF0A04C01219940CCF808156C
:108DB00003F5E0714FF0030E4CF821E0C0F80835E0
:108DC000C0F81025242202FB08F2B318C3F804905F
:108DD0002B69B350B9F1000F2FD04FF488712A7F5F
:108DE000FFF7EAFE20684FF49071FFF7E5FE206878
:108DF0004FF49271FFF7E0FE20684FF4A271FFF785
:108E0000DBFE4FF4AC712068FFF7D6FE23681A49E9
:108E1000C3F80413190B43F307335201002BD2B2EA
:108E20001CDB1648C51885F8002301225B0901F0F8
:108E30001F0102FA01F140F8231023680822C3F849
:108E40000025242303FB08660023C6E9063373616B
:108E5000012386F820303846BDE8F883084B01F03E
:108E60000F015A54E9E70827F5E71127F3E700BF98
:108E7000A0320020E98B02001003420000E100E074
:108E800014ED00E00279044B242101FB0233586900
:108E9000003818BF01207047A032002001F0604365
:108EA000B3F1005F2DE9F0470646884692463BD174
:108EB00090F80490FFF7E6FF0446002836D11D4FD6
:108EC0003068242505FB09754FF49071C5F814A08E
:108ED000C5F80880FFF770FE4FF4AC713068FFF7FB
:108EE0006BFE33686A69A968C3F84415C3F848255E
:108EF00001229A606A68DAB9D3F82021D3F85801C0
:108F00001AB90028F8D00F2007E00028FBD1012271
:108F1000DA60D3F85821002AFBD0242303FB097719
:108F200000237B61BDE8F0871020FBE71120F9E703
:108F30002046F7E7A0320020F8B501F06043B3F116
:108F4000005F04460F465ED10379304D242101FBBA
:108F50000351496821B100684FF40476C0F80863F2
:108F6000242000FB03539E6956B1D869002839D0EC
:108F700021B123684FF40472C3F80423112030E0B8
:108F80009A61DF60DE6120684FF48871FFF714FE9C
:108F900020684FF4A271FFF70FFE2368C3F8347501
:108FA000C3F8382516BB01221A602479242202FB5B
:108FB000045252680ABBD3F81011D3F84421D3F8F5
:108FC0002401114302D10028F5D00A46242303FBD3
:108FD00004550023984218BF03209A42AB6118BF82
:108FE0000F20F8BD1F61DA610126CCE7D3F800221B
:108FF00042F02002C3F80022D7E74FF40472C3F80E
:1090000004230020EDE71020EBE700BFA032002092
:1090100008B5094B1B7853B10020FFF7B5F80120C4
:10902000FFF7B2F8BDE808400320FFF7ADB8BDE890
:109030000840FFF7B5B800BFC4320020F8B57A4C3D
:10904000237805461BB100232370FFF7E1FF172D9E
:1090500000F28780DFE805F00C1717425364757F34
:10906000878C878C949999999999C3C8D0D8E3E350
:10907000FFF7CEFF6D48FDF75AFF6D4B0022044607
:109080001A702046F8BD0020FFF764F8F0B1002008
:10909000FFF77AF8022D0CBF4FF4E1644FF47A64C5
:1090A000634B1D7000254FF400464FF47A7029463B
:1090B0004FF4FA620023E4FB060102F00FF92A469E
:1090C0000146BDE8F8405948FDF719BFFFF750F8D1
:1090D000022D0CBFC8244FF4C874E1E70020FFF74D
:1090E00039F840B10020FFF74FF84FF44874504B67
:1090F00003221A70D6E7FFF73BF8C824F7E70020F1
:10910000FFF728F838B10020FFF73EF84FF47A64F3
:10911000474B0422EDE7FFF72BF84FF4C874F7E74D
:109120000020FFF717F848B10020FFF72DF8404B5B
:1091300005221A7040F6CD410022C2E7FFF718F869
:10914000F5E70020FFF74AF8394B06221A70002293
:1091500040F26661B5E70020FFF70AF8344B0722BA
:109160001A7000248DE701202070FFF737F8EEE732
:1091700001202070FFF732F800224FF40051A0E7E1
:10918000FFF71DF82A4B0C22EAE72A482A4EFDF782
:10919000CEFED5F1110504461CD0D8B9012D13D04F
:1091A000C820454321464FF400474FF47A704FF4EE
:1091B000FA620023C5FB070102F090F8224601463F
:1091C0001C48FDF79CFE04460220FEF7D1FF012358
:1091D000337056E70220FEF7D7FF0023F8E7FFF7CA
:1091E00017FF134B1222BBE7FFF712FF0020FEF719
:1091F000BFFF0F4B1322B3E7FFF70AFF0120FEF773
:10920000B7FF0B4B1422ABE7FFF702FF0020FEF77E
:10921000AFFF0120FEF7ACFF054B1522A0E7FEF7DC
:10922000CEFF034B1D709CE718330020E83200206E
:1092300019330020C8320020C432002010B50029A4
:1092400014BF03240024FEF7DBFF800000F1A040E0
:10925000D0F8002722F44032C0F80027D0F80037B9
:1092600043EA0443C0F80037002010BD044B1B68DC
:1092700013F0010301D0FFF7E1BE1846704700BFAD
:1092800014330020032811D8012A0AD101290FD153
:1092900000F10E02D2B20D4B00EB40001A54002038
:1092A00070470129F7D0022904D049B1072070473F
:1092B0000022F8E7054B00EB400018444270EEE74F
:1092C000024B00EB400018448270E8E708330020AE
:1092D000032802D80121FFF7B1BF0620704708B567
:1092E000012202210020FFF7CDFF08B1072810D18D
:1092F000072202210120FFF7C5FF08B1072808D186
:1093000000210A220846FFF7BDFF10B1072808BF59
:10931000002008BD0388102B10B502D0112B1ED0E1
:1093200010BD1A4C2168B1B901220846FFF7AAFF07
:1093300008B1072824D1072202210120FFF7A2FF4C
:1093400008B107281CD1042202210020FFF79AFF50
:1093500008B1072814D1236801332360E0E70B4AE2
:109360001368013B1360002BDAD1FFF7B8FF002828
:10937000D6D0074B1B68002BD2D0BDE81040184751
:10938000034B1B68002BE6D09847E4E7203300200E
:109390001C33002008B50020FFF79AFF08B106280B
:1093A00006D10120FFF794FF10B1062808BF002066
:1093B00008BD76DF70477ADF70477CDF70477FDF5C
:1093C00070478FDF7047B1DF704733DF7047FDF7BD
:1093D00069BC08B50020FFF749FF08B1FDF762FC42
:1093E000FFF7D8FF08B1FDF75DFCFFF7EEFF18B1FE
:1093F000BDE80840FDF756BC08BD00000388212BDE
:1094000013B504463FD007D8112B2DD0132B48D0CD
:10941000102B0CD002B010BD522B4AD0562B01D0CD
:109420003B2BF7D1A0881321FFF7C3FF15E0254B95
:1094300025482649C01AC008000440F00300FDF783
:10944000BFFA0720FFF712FF08B1FDF72BFC204BF6
:10945000A1882048198001F08DFB0028DAD002B0E5
:10946000BDE81040FDF71EBC164B17481A49C01A3C
:10947000C008000440F00300FDF7A2FA144B4FF6B9
:10948000FF721A80C6E7002380888DF8043001A996
:109490008DF80530FFF795FF0028BBD0FDF702FCE3
:1094A000B8E70B4800231A4685210088FFF787FF9D
:1094B000D3E7074800231A4619460088FFF783FFC1
:1094C000CBE700BF74B602009CB6020012BE0200D9
:1094D000062B0020683800201CBE020008B5037867
:1094E0004BB9054B3B211888FFF763FF18B1BDE866
:1094F0000840FDF7D7BB08BD062B002008B548B1D2
:1095000003280BD10220FFF7B1FE38B1BDE80840B7
:10951000FDF7C8BBBDE80840FFF75BBF08BD000012
:10952000F7B50378012B33D0022B31D073BB1B4C22
:109530001B4D20782844FDF79FFE23780133DBB2D2
:109540001D44237015F8012C0A2A05D00D2A03D0DA
:10955000144A12889A4219D8012B15D9124D104E6F
:10956000124F2378ADF806300DF106022B883146F4
:10957000384601F077FC082806D01328F1D00528DA
:1095800002D008B1FDF78EFB0023237003B0F0BDBD
:10959000406803B0BDE8F040FDF784BB18340020FC
:1095A00024330020042B0020062B0020082B002051
:1095B0002DE9F0410578064645BB154C154BDFF803
:1095C0005880E41AE408240444F00104B28A954265
:1095D0000AD33369134413F8013C0D2B16D10A202A
:1095E000FDF760FE1128F9E73369585DFDF75AFE73
:1095F000074648B11128F7D0024641462046FDF7FC
:10960000E3F93846FDF74EFB0135DFE7BDE8F081B1
:109610009CB6020074B6020029BE020038B5054DA2
:10962000044645F001054FF47A40A847013CFAD1C1
:1096300038BD00BFE0BE02000D4B4A881B889A422D
:1096400014D10A8840F677239A420FD18B88094AB1
:1096500009480A49033B9BB21380094A801AC00893
:1096600000041A4640F00300FDF7B7B9704700BF89
:10967000062B0020042B00209CB6020054BE0200E2
:1096800074B60200FDF70EBB08B50849084801F0A2
:1096900051F908B1FDF706FB0548F72101F05EF925
:1096A00018B1BDE80840FDF7FDBA08BD39960200C3
:1096B000503800204FF0A043042230B5C3F868278B
:1096C000794D0322C3F81027C3F84C274FF400222A
:1096D000C3F808250FCDB1B005AC0FC495E8030061
:1096E000724B734A01934FF4807384E80300CDE911
:1096F000032302936F4A072301A905A8FDF764FD20
:1097000008B1FDF7CFFA4FF480410020FCF7BEFF0F
:1097100008B1FDF7C7FAFCF7F7FEFDF7B3FB08B198
:10972000FDF7C0FAFEF728FB08B1FDF7BBFA01F020
:1097300015FC08B1FDF7B6FA002305A90120059331
:1097400001F09EFC08B1FDF7ADFA05A801F058FD47
:1097500008B1FDF7A7FA112357498DF804300F22FD
:1097600001A8FFF72AFE08B1FDF79CFA0023ADF827
:1097700018301023ADF814303C23ADF8163005A88E
:109780004FF4C873ADF81A30FFF715FE08B1FDF7B6
:1097900089FAFFF779FF494B4948059305A901F07C
:1097A000D7F908B1FDF77EFA464B4748019301A966
:1097B00001F0DEFA08B1FDF775FAAC22002105A828
:1097C00001F096FE02238DF8143005238DF8173032
:1097D00001234020ADF860308DF8903044F25063A2
:1097E000CDE92703394A3A4B3A48199205A92E93F5
:1097F00000F0C3FB08B1FDF755FA3648012100F02F
:10980000B9FB142200210DEB020001F071FE4FF4B0
:10981000F0234FF4A031CDE9061303238DF8203057
:109820002D4B0A9305A82D4B0B9300F063FE08B156
:10983000FDF738FA2A4801F016FE2A4B2A482B4930
:10984000C01AC008000440F00300FDF7B9F8214831
:10985000032100F00FFC08B1FDF724FA4FF0A044FB
:10986000D4F80435DA4302F0100203F01003C4F810
:1098700008254FF4FA70C4F80C35FFF7CFFED4F882
:1098800010355A01ECD540F2DC50FFF7C7FED4F892
:1098900010355B01E4D54FF40023C4F80C354FF4C8
:1098A000FA60FFF7BBFEDBE7BCBE020074380020A5
:1098B000743900202195020070BE0200CF9302008F
:1098C00068380020B1950200082B0020002B0020F2
:1098D000FD9402001C340020DD94020085960200F5
:1098E00080BE020074B602009CB6020091BE020067
:1098F0000369C26893429CBF80681B18013B981A99
:1099000070472DE9F843D0E902940546A9EB040815
:109910004068904520440F46144404D901F0BFFD2F
:10992000EC60BDE8F8834246A4EB090401F0B7FD02
:109930006868224607EB0801F0E72DE9F843C5689F
:109940000646894617464FF000083469B3687068C8
:10995000A54228BFE418013C621B5C1BBC4228BF27
:109960003C46944228BF144649462844224601F00A
:1099700096FDB3682544AB4208BF00253F1BA044B9
:10998000A144F560E1D14046BDE8F88310B5114C23
:10999000114AA2610223C4E90433104BE361A264BB
:1099A0004FF400730E4A0F492362E2640023102231
:1099B000E01DA3626362E362A3656365E3652265FC
:1099C00001F0C9FD0849204601F0C5FD2023A3711F
:1099D00010BD00BF743A0020E6BE0200FC3A002031
:1099E000EC3A0020EFBE0200F3BE020070B5164B49
:1099F000182400FB04451D4404FB00331646DC6AB2
:109A0000012C0ED0022C18D0E4B92846FFF770FFC5
:109A1000864204D832462846FFF773FF3446204674
:109A200070BD2846FFF764FF8642344628BF0446CF
:109A300022462846FFF765FFF1E72846BDE870405B
:109A4000FFF77BBF0024EAE7743A0020FFF79EBFD0
:109A50006DDF704779DF70477DDF704764DF7047E7
:109A60002DE9F04F85B000250E9CBDF83CB0B4F850
:109A700000A00191074690461E46A9463A884A45ED
:109A80000DDC45B12388013BA3EB0A039BB2FF2BFE
:109A90003AD806F80A30002005B0BDE8F08F7A68A1
:109AA00052F82900039000220DF10B0103A8FFF7E3
:109AB000D5FF0028F0D19DF80B20424521D1228806
:109AC000002D14BF0020022002EB0801014459457B
:109AD0001ADC3DB9013292B2019B2280B354228834
:109AE0000132228022880DF10B01324403A8FFF7D6
:109AF000B5FF0028D0D121889DF80B200A44228090
:109B0000012509F10109B9E70C20C5E72DE9F34169
:109B1000089FBDF824801546CDE90078022204464E
:109B20001E46FFF79DFF50B93346102229462046B6
:109B3000CDE9087802B0BDE8F041FFF791BF02B06F
:109B4000BDE8F0812DE9F04F00231788138090F8CD
:109B50002D3085B006460D4614465BB3082F01D85C
:109B60000C2028E102A8FFF773FF002840F02381B2
:109B70002388DDF809100822EA54238801339BB2B8
:109B80001B222380EA54238801339BB2EA182380E6
:109B9000E950BDF80D30938023889DF808200633E6
:109BA0009BB212F0FE0218BF01222380EA542388E0
:109BB00001332380B378FBB123880433BB42CFD871
:109BC00002A8FFF747FF002840F0F5802388032212
:109BD000EA54238801339BB219222380EA54238854
:109BE000BDF8082001339BB2E9182380EA54120A19
:109BF0004A70238802332380F2789AB12388D91CD3
:109C0000B942ADD80221E954238801339BB2012126
:109C10002380E95423880B449BB22380EA54238891
:109C20000B4423807268AAB12388D91CB94297D803
:109C3000022192F90020E954238801339BB20A21C2
:109C40002380E954238801339BB22380EA5423887C
:109C5000013323803389002B40F0A180338A5BB12C
:109C6000CDE900472B460722032106F11000FFF73C
:109C70004DFF002840F09F80338B5BB1CDE900475A
:109C80002B461522142106F11800FFF73FFF00288C
:109C900040F09180326A002A40F09080D6F824800B
:109CA000B8F1000F30D0B8F804302188981C8A1C15
:109CB0000244BA423FF654AFFE283FF651AF033399
:109CC0006B54238801339BB2FF222380EA542388FC
:109CD00001339BB22380B8F80020EA54E918120A35
:109CE0004A702088023080B22080B8F804205AB12F
:109CF000D8F8081000296BD0284401F0D0FB238845
:109D0000B8F804201344238096F82C30002B40F040
:109D10009880307800284ED03388012B58D0228884
:109D200002F1020CBC453FF61BAF012805D1737848
:109D3000023313449F42FFF413AF023FBF1ABFB276
:109D400002A905EB0C00ADF80870FFF785FE90BB8B
:109D50003178BDF80830022900F0B98072789A4253
:109D600002D39F4280F0B180012940F0B280974237
:109D700093B2C0F0AE80ADF808300821BDF80830CD
:109D8000FE2B3FF6EDAE22880133AB542288013220
:109D900092B22280A9542288134423800BE0CDE99B
:109DA00000472B460622022106F10800FFF7AEFE0F
:109DB00000283FF453AF05B0BDE8F08FB4F800C001
:109DC0000CF10603BB423FF6CBAE1188052901D842
:109DD0000720F0E76FF4486E01EB0E039BB24FF2E1
:109DE0007D3E7345F4D95388052BF1D96FF4486053
:109DF000181880B27045EBD94FF6FF70814201D040
:109E00009942E5D8052305F80C30238801339BB22D
:109E100012212380E954238801339BB223801188C7
:109E2000E954E818090A4170238802339BB2238061
:109E30005288EA54E918120A4A70238802332380B0
:109E40002CE7B36A002BC3D04FF000084FF00C0A88
:109E50004FF0160BB16A5FFA88F20AFB02F201EBCF
:109E60000209B9F80430981CFE283FF679AE208824
:109E700003332B54238801339BB2238005F803B0AE
:109E8000238801339BB223808A5AEA54E918120AC4
:109E90004A702088023080B22080B9F804205AB17C
:109EA000D9F80810002993D0284401F0F8FA238843
:109EB000B9F804201344238096F82C2008F10108F7
:109EC0005FFA88F39A42C5D823E7092156E79F42F3
:109ED000FBD2ADF8087050E730B5C8B1F2B100243C
:109EE000651C8D4206DA1588A54212D805196D78D1
:109EF0009D420ED1A14211D9005D48B1013880B216
:109F000030B10234A3B210FA84F4A14206DB13800C
:109F100030BD055D01352C44A4B2E1E70020F7E730
:109F200013B513460022ADF806200DF106020446D3
:109F3000FFF7D2FF10B1BDF80630E01802B010BD37
:109F400072DF704773DF704738B5012204460D4653
:109F5000B0F81414D0F81004FFF7E2FF00B1057058
:109F600004F13C0204F5826104F15400BDE838407C
:109F7000FFF7E6BF80F830107047F8B504460F468B
:109F8000002973D0002871D091F87A301BB191F874
:109F90009830002B6CD1D7F8A030042B68D0D7F8BC
:109FA0009C30042B64D04FF0000C84F802C007F101
:109FB00078060FCE251D0FC50FCE0FC596E80700FA
:109FC00085E8070084F830C0D7F8A4306363D7F879
:109FD000A830A36304F582624FF6FF73C4F826C469
:109FE000A4F82434C4F82024C4F829C422780AB977
:109FF00084F8543094F82430002B14BFEE231F2330
:10A0000004F15501C4F81014A4F8143404F21442F5
:10A010003846FFF797FD40BB94F82430002B14BF5F
:10A02000EE231F2304F23121C4F81814A4F81C34C1
:10A0300004F21C4207F13C00FFF784FDA8B9A369B4
:10A04000A4F848304FF480730125A4F850306369B8
:10A050002064014684F83C50636404F13C0204F13E
:10A060005400FFF76DFF00B92570F8BD0E20FCE726
:10A070000720FAE7F8B5077804460D46002F00F0F0
:10A0800001810023C0F82634C0F82934C3888170C8
:10A0900000F226460BB1012903D0E37943B1022D2A
:10A0A00006D1636BABB1012284F82D2408209847B8
:10A0B00004F2274304F22D4113F8012B12B99942FF
:10A0C000FAD117466B1E032B4ED8DFE803F0050BC1
:10A0D0000F1284F82D34EBE7A3791BB194F82430E8
:10A0E00003B95FB9E3790BB1002F3FD1237A002B7D
:10A0F0003ED1637A002B0CBF00250425636BA5704D
:10A10000002B37D0033D012D34D8627992B394F8F7
:10A110002E247ABB84F83024012284F82F240720CF
:10A12000984704F13C0518220021284601F0E0F987
:10A13000E26A531E0121022B28BF0A4684F85120EF
:10A1400094F8242084F83C1032B1A36A581E0228E7
:10A1500028BF0B4684F85230A378042B1CD8DFE8C4
:10A1600003F0780D23365A000025C7E70225C5E71E
:10A170000325C3E7002384F82F34D2E7012384F8B2
:10A1800031300023C4E91063C4F82034022384F87A
:10A190003C308023A4F84830A378002B5DD1636B5A
:10A1A000002B6BD1002068E00223002A84F83130B4
:10A1B00014BF0723032384F83C302369A4F84830F4
:10A1C0000023C4F82034E36826646364E4E7636929
:10A1D0006364A369A4F8483012B1062384F83C30C4
:10A1E0006379B3B194F82E349BB994F8303483B1C9
:10A1F000022384F8503004212046FFF7A5FE0028F2
:10A20000CAD1052384F8313004F58263C4F82034C0
:10A21000C2E70323F6E7E3696364236AA4F84830DE
:10A2200012B1062384F83C30637983B194F82E345C
:10A230006BB994F8303453B1022384F850300421C0
:10A240002046FFF781FE0028A6D10623DAE7042383
:10A25000D8E7002384F831309EE7D4F820142A464A
:10A2600004F15400FFF76CFE38B994F8301094F8FC
:10A270005400FFF767FE002891D0F8BD94F8310034
:10A2800098478FE70820F8E70388112B10B50C4694
:10A290000AD0262B1FD0102B05D1C37B012B02D156
:10A2A0008388A1F8243410BD0022838881F82E24ED
:10A2B000B1F824249A42F6D10B79002BF3D1012175
:10A2C0002046FFF7D7FE0028EDD0A36B002BEAD085
:10A2D000BDE810401847037A013B012BE3D8897889
:10A2E00005230131B1FBF3F303EB8303C91AC9B2B0
:10A2F000E6E775DF704776DF70477ADF70477BDF10
:10A3000070470000034B1A8882420CBF1846002099
:10A31000704700BF183D0020024B9B6903B11847EE
:10A32000704700BFFC3C002073B585B22846FFF79C
:10A33000E9FF044638B3174E027A337B9A420CD2B7
:10A3400000F10A012846FFF7D4FFF0B111281AD016
:10A3500002B0BDE87040FFF7DFBF00230372337C1B
:10A3600043B13B212846FFF7C6FF30F0080301D078
:10A37000FFF7D2FF736933B100228DF80420ADF8E6
:10A38000065001A8984702B070BD237A01332372AA
:10A39000F9E700BFFC3C002037B50B46497A0F4A6D
:10A3A00079B9D2E901141D7A0246002D18BF214661
:10A3B0005868FCF7A4FD78B103B0BDE83040FFF762
:10A3C000ABBF00211972536933B10122ADF8060009
:10A3D0008DF8042001A8984703B030BDFC3C002054
:10A3E0004B8802889A4212D842889A420FD38088BA
:10A3F0008B8840F2F311884294BF021A421A9A42A3
:10A4000005D80844984234BF00200120704700203E
:10A41000704700000388122B70B5014659D004D84C
:10A42000102B1ED0112B44D070BD502BFCD12F4BC4
:10A43000C288DB899A42F7D1038A022BF4D186883D
:10A440003046FFF75FFF05460028EDD001F112000E
:10A4500000F07FF938BB6868FCF769FD0028E3D09D
:10A4600009E0C37B012BDFD14FF6FF70FFF74AFFF6
:10A47000054620B90420BDE87040FFF74DBF1C4AD7
:10A480008E880680002303721368C0F80A30536870
:10A49000C0F80E3010310A30FFF7A2FF134B68727C
:10A4A000DB89002BC0D129463046BDE87040FFF75C
:10A4B00073BF8088FFF726FF04460028B4D04068A9
:10A4C000FCF735FD08B1FFF727FF4FF6FF73238038
:10A4D000AAE786883046FFF715FF05460028A3D077
:10A4E00008310A30FFF77CFF6872DCE7FC3C002093
:10A4F0002C3D0020F8B5064648B305460FCD154F54
:10A500003C460FC495E8070084E807003068124C09
:10A510003C60B0B1FFF7F1FEC0B932681368236048
:10A52000536863600D480E4A4FF6FF7303800D4B6E
:10A5300040F8043F0021FCF7D7FC002818BF032097
:10A5400004E02046FFF7DBFE0028EBD0F8BD0E202C
:10A55000FCE700BFFC3C00202C3D0020183D002003
:10A5600029A30200383D00200AB1FDF7C3B8FDF76A
:10A57000CAB873B50191019C06466CB100252C4602
:10A58000294601A8FDF7C9F818B106EB44030134C8
:10A590009D800135142DF3D13046346002B070BD7A
:10A5A0002DE9F04703888488103B8CB005460A2BC0
:10A5B00021D8DFE803F0064020202020202020655D
:10A5C0004700DFF8E880D8F80830DB430093D8F87C
:10A5D00004106846FDF7CDF8009901A8FFF7C9FF00
:10A5E0000DF108090027019B9F4207D3132C12D9B4
:10A5F0000420FCF757FB0CB0BDE8F08739F802AB3C
:10A6000000260136514608EB8600FDF77CF81E2E29
:10A61000F7D10137E7E71F482146FDF76BF81E48E1
:10A620002146FDF767F8EB7B022BE4D11B4821465E
:10A63000FDF760F8DFE7174821460CB0BDE8F047AA
:10A64000FDF761B8027A16483F2A4FEA12152146F3
:10A6500094BF00220122FFF787FF022D94BF002242
:10A66000012210482146FFF77FFF012D0E4894BFBD
:10A670000022012221460CB0BDE8F047FFF774BF6D
:10A68000037A002BB7D1427A0548C2F3C0022146B3
:10A69000F1E700BF603D00205C3D0020643D0020EC
:10A6A000703D00206C3D0020683D0020583D00209A
:10A6B0001328014602D80248FDF72FB80020704742
:10A6C0005C3D002010B50446FFF7F2FF002814BFE0
:10A6D0002046142010BD70B50546164608460AB936
:10A6E0000E2070BD00231360002DF9D02B68002BC5
:10A6F000F6D0EB8813F003040ED1FFF7E3FFC0B2EE
:10A7000014280BD02B7983420AD9EA882B6800FBE6
:10A71000023030602046E4E70720E2E70520E0E76A
:10A720000420DEE7AADF7047002301380B700428FD
:10A7300006D8DFE800F00306080A0C0011230B70AE
:10A7400070472123FBE73123F9E71223F7E72223A0
:10A75000F5E7008800F001007047F0B58B7891B004
:10A760000C46012B38BF012300278DF80E3005461B
:10A770000B88607CADF80C306946ADF800708DF840
:10A780000270FFF7D1FFA07C0DF10101FFF7CCFFB4
:10A790001646237BE27B217D43EAC203227C43EA07
:10A7A00002139DF80220B94222F0190203F01903A6
:10A7B00014BF02210121134361F342031C223946D5
:10A7C00009A88DF8023000F093FE637B13F0300F80
:10A7D00014D00DF10901E07CADF808708DF80A7015
:10A7E000FFF7A2FF11238DF808309DF80A300121F0
:10A7F00002AA61F342038DF80A300E92637B8DF852
:10A800002430A37B8DF825300023CDE9063308934F
:10A8100003AB0493A388ADF81C30A368CDF814D023
:10A820001BB1E288ADF818200893A36973B301A99E
:10A830000022ADF804208A701A88ADF82C205A88BE
:10A84000ADF82E205A680D91187B0A92FFF76CFF25
:10A85000A3690DF10501587BFFF766FFA3699A7A9A
:10A86000197A41EAC201DA7A9B7B41EA02119DF82A
:10A870000620002B01F0190122F0190214BF022357
:10A880000123114363F342018DF80610E36903B11C
:10A890000C93334604AA09A92846FFF743FF11B0D9
:10A8A000F0BD90DF7047A5DF7047B5DF704700004F
:10A8B0007FB50023ADF80810ADF80A106A4602A96A
:10A8C0000646ADF80C30ADF80E300093ADF804300C
:10A8D000FFF7E7FF054600B3114B124CE41AE408FA
:10A8E000FDF7C4FA240444F0010403460E4932463D
:10A8F0002046FCF772F8BDF80020BDF8023052EA9D
:10A90000030103D009492046FCF767F8BDF804208D
:10A910001AB107492046FCF757F8284604B070BD25
:10A9200074B60200C4B60200FABE020044BF0200C0
:10A9300083BF020080B14FF0F7130360FB23037164
:10A94000F723C3801723038141F6FB320023016103
:10A9500043818281184670470E20704730B1A1F1C3
:10A960001703E02B04D80180002070470E207047A9
:10A970000720704713B5034680880C46B8B91A887B
:10A98000242A00F09C8014D8112A74D0232A00F0C5
:10A99000A780102A3ED0A37A4BB1E1880020FFF7B0
:10A9A00082FF002840F0A2804FF48073638102B0E0
:10A9B00010BD3A2A68D0552AEDD1DB88C988A0722B
:10A9C000172B38BF17238B4228BF0B462381FFF775
:10A9D0006CFF60B1FDF74AFA4E4B4F4902464F48B3
:10A9E0001B1ADB081B0443F00100FBF7EDFFE27AC2
:10A9F000002AD0D12369002BCDD040F67721ADF8C5
:10AA000002202289ADF80010ADF8042069462046E6
:10AA10009847C0E7DB7B0A790A73012B13D0022B1E
:10AA200014D0E18823898B4205D20020FFF73BFF39
:10AA300070B90123E372217B637B8B42ABD2002090
:10AA4000FFF736FFA7E70B88E380EAE74B88FBE7D1
:10AA5000112802D10123A372EDE7FDF707FA2D4B70
:10AA60002F4902462D481B1ADB081B0443F0010046
:10AA7000FBF7AAFFDFE7F723CB8017230B8141F613
:10AA8000FB3348818B8186E75B89CA88934228BF64
:10AA90001346172B0A6938BF17230B8162B1C97A95
:10AAA00051B140F67721ADF80010ADF80200ADF8D5
:10AAB0000430694620469047002363816BE71A7A89
:10AAC0000B694A73002B3FF466AF4DF67A218DF87F
:10AAD0000500ADF80010ADF802008DF8042095E7F0
:10AAE000197A237B994228BF1946A9E711283FF418
:10AAF0005EAFFDF7BBF9074B0949024607481B1A31
:10AB0000DB081B0443F0010002B0BDE81040FBF776
:10AB10005BBF00BFC4B602000AC0020074B60200E8
:10AB2000D9BF0200B0DF704766DF704710B5002163
:10AB300004464088FFF7F8FF034608B9237210BDAA
:10AB4000112801D10123F9E76368BDE810401847D7
:10AB500060B159B10378DE2B0AD00B684360DE2365
:10AB600003704FF6FF734380002070470E2070473C
:10AB70000820704728B10378DE2B04D141800020E3
:10AB800070470E20704708207047F0B5054685B025
:10AB90000C46002942D0002840D00B78DE2B3DD156
:10ABA00082884B889A4204D10B7A13B10846FFF78A
:10ABB000BDFF2B88112B33D0512B0FD0012B2DD162
:10ABC0002B7A012B2AD1A9886288914226D120466E
:10ABD000237205B0BDE8F040FFF7A8BFAE886388D8
:10ABE000B3421BD1AF79022F18D1AD7B2B1F022BA3
:10ABF00014D800211022684600F07AFC052D18BFF9
:10AC00004FF4C0736946304618BFADF804308DF874
:10AC10000070FFF787FF08B16368984705B0F0BD83
:10AC20006388AA889A4204BF4FF6FF736380F5E7F2
:10AC3000A8DF7047ADDF7047AEDF704762DF704757
:10AC4000F0B505468BB00C4600295FD000285DD0DA
:10AC50000388502B35D0572B6CD0102B56D18188C0
:10AC60006069002601AA0196FFF735FD02232189BC
:10AC7000A888ADF80A6002AACDF80CD0ADF808306B
:10AC8000FFF7D8FF002841D1A369002B3ED00398DD
:10AC9000FFF75FFD002839D0019E0EB1012333700C
:10ACA0001822002104A800F023FC02238DF81030A4
:10ACB000AB88ADF81830A3690594079604A89847A7
:10ACC00024E08188606902AAFFF705FD18220021AF
:10ACD00004A800F00DFCAB882189ADF81830EB8892
:10ACE000029A05949942079217D12E8A022E14D106
:10ACF00062B105F11200FFF72CFD029B40B1012269
:10AD00001A708DF81060A369002BD7D10BB0F0BD7D
:10AD1000187003238DF81030F5E7A2899A42F5D117
:10AD2000A369002BF2D005F1120208922A8AADF82D
:10AD30002420C3E78188606902AAFFF7CCFC0146A2
:10AD40000028E3D1029F3B78002BDFD0A669002EBC
:10AD5000DCD0182204A800F0CBFB01238DF81030C2
:10AD6000AB880594ADF81830079704A8B047CDE735
:10AD7000F0B53A4B8FB002AD04460A4603F1100C11
:10AD80002F46186859682E4603C608336345354672
:10AD9000F7D1002C5FD0002A5DD01368A361214653
:10ADA0003846FFF74BFF002853D12246012512F801
:10ADB000023B8DF8063001A92846ADF80450FFF794
:10ADC00037FF002845D10146202206A800F090FB5D
:10ADD00022460223ADF8183012F80C3B8DF81A30D9
:10ADE000BDF824301E4E6088079623F44F6323F08D
:10ADF0000F0343F440632B4306A9ADF824308DF8CC
:10AE000029508DF82A50FFF7A8FC10BB01462022DC
:10AE100006A800F06DFB22460323ADF8183012F8A7
:10AE2000043B8DF81A30BDF824306088079623F46F
:10AE3000875323F01F0343F480532B43ADF8243092
:10AE400006A940F201138DF82950ADF82A30FFF71A
:10AE500084FC0FB0F0BD0E20FBE700BF4EC0020027
:10AE6000F4000100F0B50F4687B016461C460546B3
:10AE700010B3406901AA1946FFF72DFCD0B94FF66F
:10AE8000FF739C421AD0019BC3B11B78C3B13388B6
:10AE9000F42B17D8AB88CDF80B008DF80F00ADF868
:10AEA000083002A901232046CDE904678DF80A3055
:10AEB000FFF7C2FE07B0F0BD0E20FBE70520F9E763
:10AEC0000820F7E70720F5E710DF704713B50446C1
:10AED00009496846FCF76FFF019808B902B010BD38
:10AEE000D0E900212046904718B16846FCF76DFF75
:10AEF000F2E71120F2E700BF6CC0020013B5044670
:10AF000007496846FCF757FF019B0BB902B010BD1B
:10AF10002046D3E9002190476846FCF756FFF3E747
:10AF200084C002000B4991F816335A09EC231341EF
:10AF3000DB0706D5084B9A683AB94FF480030B60DB
:10AF4000704742F20200FBF7ADBE1A6842F480027D
:10AF50001A60704700E100E0C0310020F7B5194FDA
:10AF60003C7864BB184E012520463570FFF7AEFFD4
:10AF7000112821D02046FFF7C1FF144B8DF8034064
:10AF8000186801900DF10300FCF7B4F9104901A80D
:10AF9000FFF79AFF0446B0FA80F0400938709DF838
:10AFA0000300FCF7CBF93CB90A4B34701C70FFF777
:10AFB000B9FF2846FFF7A2FF204603B0F0BD0824E2
:10AFC000FAE700BFD53D0020D43D002066C0020056
:10AFD000C16C0200D63D0020014B1878704700BFBD
:10AFE000D53D002007B508496846FCF7E4FE019B03
:10AFF00013B903B05DF804FBD3E90020904768461D
:10B00000FCF7E3FEF3E700BF78C00200FFF7EABFFA
:10B0100060DF704769DF704761DF704730B5134DFF
:10B02000ADF5017D4FF4FA740DF1020103A8ADF8FE
:10B030000240FFF7F1FF70B9294601A8FCF7BBFEFB
:10B04000029B002BF0D003A8D3E90021904701A870
:10B05000FCF7BBFEF4E7052805D00DF5017DBDE842
:10B060003040FBF71FBE0DF5017D30BD0CC3020063
:10B07000024B1B780BB1FFF7D1BF7047D73D0020C3
:10B0800030B5054685B00C46002900F0A4800023A9
:10B09000CDE90133514A039301230A608DF804007E
:10B0A0008DF8063001A906232020ADF80830FFF7FF
:10B0B000B1FF60B1FCF7DAFE494B4A4902464A4803
:10B0C0001B1ADB081B0443F00100FBF77DFC002387
:10B0D000CDE9013303932268012301A940208DF8B3
:10B0E0000530FFF797FF60B1FCF7C0FE3C4B3F49CE
:10B0F00002463D481B1ADB081B0443F00100FBF726
:10B1000063FC0023CDE90133039322688DF80450DA
:10B11000F72301A92320ADF80630FFF77BFF60B1CC
:10B12000FCF7A4FE2E4B324902462F481B1ADB08BF
:10B130001B0443F00100FBF747FC002301202268B9
:10B14000039301A9CDE901338DF80400FFF762FFF5
:10B1500060B1FCF78BFE224B2649024622481B1A9F
:10B16000DB081B0443F00100FBF72EFC0023CDE9B4
:10B17000023322684FF4B06301A9A1200193FFF7C5
:10B1800049FF60B1FCF772FE154B1B490246164899
:10B190001B1ADB081B0443F00100FBF715FC00251C
:10B1A0002268039501A9A020CDE90155FFF732FFE0
:10B1B000034668B1FCF75AFE094B104902460A489B
:10B1C0001B1ADB081B0443F00100FBF7FDFB2B46B9
:10B1D000184605B030BD0E23FAE700BFD82A00207C
:10B1E000D4B6020090C0020074B60200D6C00200BD
:10B1F00022C1020069C10200B5C1020006C20200FC
:10B2000073B505460668FFF703FF2B68B342044693
:10B210001DD91A481A4B1B491B1ADB081B0443F0A3
:10B2200002000190FBF7CCFB2B68174901983246CE
:10B23000FBF7D3FB4FF080532A68D3F80C31134946
:10B2400001989B0203F100539A1AFBF7BDFB2CB93E
:10B250000F4B01221A70204602B070BD2046FCF749
:10B2600005FE074B0B49024604481B1ADB081B046A
:10B2700043F00100FBF7A8FBEDE700BF74B6020046
:10B28000D4B6020059C2020088C20200B9C202004C
:10B29000D73D0020E3C202004BDF70471FB50E4CC4
:10B2A00001A8FFF7F9FF70B9214602A8FCF783FD5A
:10B2B000039B002BF4D00198D3E90021904702A80A
:10B2C000FCF783FDF4E7052804D004B0BDE8104086
:10B2D000FBF7E8BC04B010BD24C3020053EA020C23
:10B2E00061D02DE9F04BB3FA83F51E0007BFB2FA27
:10B2F00082F502FA05F403FA05F41646C5F12005B5
:10B300001EBF22FA05F73C43203556EA044C4FEAAB
:10B31000144418BF0134A3464FF00009C8469042B8
:10B3200071EB030C39D3094207BFB0FA80F700FA7A
:10B3300007F6B1FA81F701FA07F6C7F120071EBF39
:10B3400020FA07FC46EA0C062037B6FBFBFC7F1B05
:10B35000103F07F01F04C4F120060CFA04F42CFA85
:10B3600006F644BF34460026202FA4BF26460024FC
:10B3700054EA060C08BF012418EB040849EB06093F
:10B38000A4FB027CC01B06FB02CC04FB03CC71EBCC
:10B390000C01904271EB030CC5D20B4602464946A4
:10B3A0004046BDE8F08BB2FBF3F200007F2805D8E1
:10B3B000034B185C034B5B5C1840704700207047E0
:10B3C0003CC30200BCC30200A0F16103192B98BF6B
:10B3D00020387047A0F14103192B98BF20307047E7
:10B3E0007F2805D8034B185C034B5B5C1840704703
:10B3F000002070473CC30200BCC30200A0F16103FF
:10B40000192B98BF20387047A0F14103192B98BF22
:10B41000203070477F299ABF017001206FF02E0005
:10B4200070475AB10A787F2A0AD800B10260002119
:10B4300019605960501A18BF0120704700207047EA
:10B440006FF02E007047000008B5034B5B689B68E7
:10B450001B68984708BD00BF2C2B002008B50921A8
:10B46000FFF7F2FF08BD70B5054600F0C6F8013DD4
:10B47000002615F8010F48B13146FCF701FD0446DE
:10B48000B0F1FF3FF5D100F0B9F806E000210A2045
:10B49000FCF7F6FC044600F0B1F8204670BD844687
:10B4A00040EA010313F0030F18D18446202A0BD37E
:10B4B0002DE9F007B1E8F807A0E8F807A2F12002AB
:10B4C000202AF7D2BDE8F007042A07D351F8043B3D
:10B4D00040F8043BA2F10402042AF7D2002A05D066
:10B4E00011F8013B00F8013B013AF9D16046704781
:10B4F0008446002A2DD010F0030F04D000F8011B61
:10B50000013A26D0F7E7C9B241EA012141EA0141F7
:10B51000202A12D3A2F120022DE9F0030B460C469B
:10B520000D460E460F4688468946A0E8FA03203AA3
:10B53000FBD2BDE8F00320320BD0042A05D340F83B
:10B54000041B043A05D0042AF9D200F8011B013A81
:10B55000FBD160467047024610F0030F16D111F080
:10B56000030F13D12DE9F0004FF001374FF0803376
:10B5700051F8044BA4EB070525EA04051D4002D150
:10B5800042F8044BF4E7A1F10401F0BC11F8013BCF
:10B5900002F8013B002BF9D1704700F1010110F0D6
:10B5A000030F11D010F8012B002A23D010F0030F45
:10B5B0000AD010F8012B002A1CD010F0030F03D082
:10B5C00010F8012B002A15D02DE970004FF0013240
:10B5D0004FF0803350F8044BA4EB020525EA040534
:10B5E0001D4000D1F6E7A0F1040070BC10F8012B5B
:0EB5F000002AFBD1A0EB0100704770477047A6
:08B600004D8202000000000071
:10B60800A1A5020000000000159302000000000040
:10B6180089A202001C34002075A9020050380020BD
:10B6280015A40200000000008BAB0200683800205F
:10B6380041AC0200082B0020FD930200000000002E
:08B64800E9820200000000008D
:10B6500071B00200000000009DB202000000000076
:10B66000842B00204C2C0020542C00208C2B0020FC
:04B6700018000000BE
:10B67400F6BD020000000000FCBD02000000000056
:10B6840003BE02000000000007BE0200000000002C
:10B694000CBE02000000000045B7020000000303D6
:10B6A4001CB802000000000040B8020000000000C6
:10B6B40046C0020000000000F0BD020000000000CF
:10B6C40039C00200000003035EC00200000003034F
:10B6D40000C302000000030318C3020000000303B8
:10B6E400C6B8020000000000DCB802000000000040
:10B6F40018B702000000000024B70200D82A002076
:10B704000000000000000000000000000338FDD825
:10B7140070470000D563020041640200D163020057
:10B724007274745F6C6F675F6261636B656E6400F3
:10B734004261636B656E647320666C7573686564DF
:10B744000061707000000000743000207F00000071
:10B75400F43000201B5B313B33316D0025734C6F9B
:10B7640067732064726F70706564202825642925CE
:10B77400730D0A001B5B306D002573003C25733E7E
:10B784002025733A20002025303278002020200024
:10B794007C002563001B5B313B33306D001B5B3148
:10B7A4003B33326D001B5B313B33336D001B5B312C
:10B7B4003B33346D001B5B313B33356D001B5B3118
:10B7C4003B33366D001B5B313B33376D0077617261
:10B7D4006E696E6700696E666F0064656275670006
:10B7E40078B7020099B7020058B70200A1B7020067
:10B7F400A9B70200B1B70200B9B70200C1B702008D
:10B80400C9B70200000000002DB80200D1B7020041
:10B81400D9B70200DEB702006170705F627574749C
:10B824006F6E00466174616C206572726F720053B2
:10B83400797374656D207265736574006170705FEF
:10B8440074696D65720001000600000000000000CC
:10B854000C310020916D0200FFFFFFFFFFFFFFFF8F
:10B86400FFFFFFFFFFFFFFFF0000000000000000DC
:10B874000000D6010601000052544320696E73741F
:10B88400616E636520616C726561647920696E69BB
:10B894007469616C697A65642E005254433A206974
:10B8A4006E697469616C697A65642E000338FDD829
:10B8B40070473031323334353637383941424344B6
:10B8C40045467077725F6D676D74000048B602007C
:10B8D40048B6020004000000736F72746C697374DC
:10B8E400004E52465F53554343455353004E524610
:10B8F4005F4552524F525F5356435F48414E444C4A
:10B9040045525F4D495353494E47004E52465F4599
:10B9140052524F525F534F46544445564943455F34
:10B924004E4F545F454E41424C4544004E52465F93
:10B934004552524F525F494E5445524E414C004E6F
:10B9440052465F4552524F525F4E4F5F4D454D0038
:10B954004E52465F4552524F525F4E4F545F464FD0
:10B96400554E44004E52465F4552524F525F4E4F21
:10B97400545F535550504F52544544004E52465F05
:10B984004552524F525F494E56414C49445F5041D3
:10B9940052414D004E52465F4552524F525F494EFE
:10B9A40056414C49445F5354415445004E52465FFE
:10B9B4004552524F525F494E56414C49445F4C45A3
:10B9C4004E475448004E52465F4552524F525F49CB
:10B9D4004E56414C49445F464C414753004E5246F3
:10B9E4005F4552524F525F494E56414C49445F4461
:10B9F400415441004E52465F4552524F525F4441BA
:10BA040054415F53495A45004E52465F4552524F86
:10BA1400525F54494D454F5554004E52465F45526E
:10BA2400524F525F4E554C4C004E52465F45525257
:10BA34004F525F464F5242494444454E004E52468F
:10BA44005F4552524F525F494E56414C49445F4103
:10BA5400444452004E52465F4552524F525F425543
:10BA64005359004E52465F4552524F525F434F4E18
:10BA74004E5F434F554E54004E52465F4552524F0F
:10BA8400525F5245534F5552434553004E52465F01
:10BA94004552524F525F4D4F44554C455F4E4F54A3
:10BAA4005F494E495449414C495A4544004E524617
:10BAB4005F4552524F525F4D555445585F494E4968
:10BAC400545F4641494C4544004E52465F455252EC
:10BAD4004F525F4D555445585F4C4F434B5F464161
:10BAE400494C4544004E52465F4552524F525F4DB9
:10BAF400555445585F554E4C4F434B5F4641494C56
:10BB04004544004E52465F4552524F525F4D555484
:10BB140045585F434F4E445F494E49545F4641493F
:10BB24004C4544004E52465F4552524F525F4D4F72
:10BB340044554C455F414C52454144595F494E4937
:10BB44005449414C495A4544004E52465F4552526D
:10BB54004F525F53544F524147455F46554C4C003A
:10BB64004E52465F4552524F525F4150495F4E4FCD
:10BB7400545F494D504C454D454E544544004E523A
:10BB8400465F4552524F525F464541545552455FB8
:10BB94004E4F545F454E41424C4544004E52465F21
:10BBA4004552524F525F494F5F50454E44494E47AC
:10BBB400004E52465F4552524F525F4452565F54B4
:10BBC40057495F4552525F4F56455252554E004EAB
:10BBD40052465F4552524F525F4452565F54574942
:10BBE4005F4552525F414E41434B004E52465F45C2
:10BBF40052524F525F4452565F5457495F45525216
:10BC04005F444E41434B004E52465F4552524F52A1
:10BC14005F424C455F495053505F52585F504B54FC
:10BC24005F5452554E4341544544004E52465F457D
:10BC340052524F525F424C455F495053505F434804
:10BC4400414E4E454C5F414C52454144595F455825
:10BC540049535453004E52465F4552524F525F422D
:10BC64004C455F495053505F4C494E4B5F444953D8
:10BC7400434F4E4E4543544544004E52465F455251
:10BC8400524F525F424C455F495053505F504545B7
:10BC9400525F52454A454354454400556E6B6E6F9E
:10BCA400776E206572726F7220636F6465000000A6
:10BCB40000000000E5B8020001000000F1B8020035
:10BCC400020000000FB902000300000030B90200B6
:10BCD4000400000043B902000500000054B902004A
:10BCE4000600000068B902000700000080B90200E5
:10BCF4000800000098B9020009000000B0B9020071
:10BD04000A000000C9B902000B000000E1B90200FA
:10BD14000C000000F8B902000D0000000CBA02008B
:10BD24000E0000001EBA02000F0000002DBA02002F
:10BD34001000000041BA02001100000058BA0200CD
:10BD44001200000067BA0200130000007CBA02006F
:10BD54008000000090BA020081000000B1BA020025
:10BD640082000000CDBA020083000000E9BA02009C
:10BD74008400000007BB02008500000028BB02000D
:10BD8400860000004DBB02009000000064BB02006E
:10BD94009100000082BB020092000000A0BB0200E0
:10BDA40000820000B5BB020001820000D3BB020088
:10BDB40002820000EFBB0200008400000BBC020002
:10BDC400018400002FBC02000284000059BC020060
:10BDD400038400007EBC0200000001010000000199
:10BDE400010000000D0E0F1011121314636C6F6329
:10BDF4006B00434C4F434B004750494F5445005050
:10BE04005253005541525400554152544500436F1A
:10BE14006E6E656374656400446973636F6E6E650A
:10BE240063746564004661696C656420726563656A
:10BE34006976696E67204E5553206D65737361672B
:10BE4400652E204572726F7220307825782E20007E
:10BE540044617461206C656E20697320736574207D
:10BE6400746F203078255828256429004E6F726439
:10BE740069635F554152545F454D47000D0A554172
:10BE8400525420737461727465642E0D00446562AB
:10BE94007567206C6F6767696E6720666F722055DF
:10BEA400415254206F766572205254542073746149
:10BEB400727465642E000000080000000600000093
:10BEC40005000000070000000000000000E0D701AA
:10BED4000000000000000000000000000338FDD84E
:10BEE40070475465726D696E616C0052545400530E
:10BEF40045474745520073645F626C655F676170D4
:10BF04005F646174615F6C656E6774685F757064AB
:10BF140061746528292028726571756573742920F8
:10BF24006F6E20636F6E6E656374696F6E20307818
:10BF340025782072657475726E65642025732E00F1
:10BF4400546865207265717565737465642054580E
:10BF54002F5258207061636B6574206C656E677432
:10BF64006820697320746F6F206C6F6E672062792C
:10BF74002025752F2575206F63746574732E005406
:10BF840068652072657175657374656420636F6D8F
:10BF940062696E6174696F6E206F66205458206107
:10BFA4006E64205258207061636B6574206C656EFA
:10BFB4006774687320697320746F6F206C6F6E6789
:10BFC400206279202575206D6963726F7365636FD4
:10BFD4006E64732E0073645F626C655F6761747472
:10BFE400635F65786368616E67655F6D74755F72C2
:10BFF40065717565737428292072657475726E6530
:10C00400642025732E0073645F626C655F676174DE
:10C0140074735F65786368616E67655F6D74755F7F
:10C024007265706C7928292072657475726E656406
:10C034002025732E006E72665F626C655F676174A3
:10C044007400626C655F6E7573009ECADC240EE535
:10C05400A9E093F3A3B50000406E6E72665F73644B
:10C06400680001000007000048B6020048B602005C
:10C074000800000050B6020060B60200080000008C
:10C0840048B6020050B602000800000073645F6204
:10C094006C655F6366675F736574282920726574D5
:10C0A40075726E6564202573207768656E206174EF
:10C0B40074656D7074696E6720746F207365742085
:10C0C400424C455F434F4E4E5F4346475F474150A6
:10C0D4002E0073645F626C655F6366675F7365748B
:10C0E40028292072657475726E6564202573207723
:10C0F40068656E20617474656D7074696E67207410
:10C104006F2073657420424C455F4741505F43463E
:10C11400475F524F4C455F434F554E542E00736456
:10C124005F626C655F6366675F736574282920725C
:10C13400657475726E6564202573207768656E205A
:10C14400617474656D7074696E6720746F207365B3
:10C154007420424C455F434F4E4E5F4346475F4712
:10C164004154542E0073645F626C655F6366675F5D
:10C1740073657428292072657475726E6564202550
:10C1840073207768656E20617474656D7074696E70
:10C194006720746F2073657420424C455F434F4D94
:10C1A4004D4F4E5F4346475F56535F555549442EA6
:10C1B4000073645F626C655F6366675F73657428B0
:10C1C400292072657475726E656420257320776802
:10C1D400656E20617474656D7074696E6720746F28
:10C1E4002073657420424C455F47415454535F4368
:10C1F40046475F415454525F5441425F53495A4544
:10C204002E0073645F626C655F6366675F73657459
:10C2140028292072657475726E65642025732077F1
:10C2240068656E20617474656D7074696E672074DE
:10C234006F2073657420424C455F47415454535FEB
:10C244004346475F534552564943455F4348414E31
:10C254004745442E00496E73756666696369656E69
:10C26400742052414D20616C6C6F6361746564206D
:10C27400666F722074686520536F667444657669CE
:10C2840063652E004368616E67652074686520529B
:10C29400414D207374617274206C6F636174696FB3
:10C2A4006E2066726F6D203078257820746F203090
:10C2B4007825782E004D6178696D756D2052414D59
:10C2C4002073697A6520666F72206170706C69638F
:10C2D4006174696F6E20697320307825782E00733D
:10C2E400645F626C655F656E61626C6528292072AB
:10C2F400657475726E65642025732E006E72665FB8
:10C304007364685F626C650008B6020048B6020098
:10C31400080000006E72665F7364685F736F630089
:10C3240000B6020008B60200080000004300000046
:10C33400504F534958000000202020202020202066
:10C344002068282828282020202020202020202081
:10C354002020202020202020481010101010101021
:10C364001010101010101010848484848484848429
:10C37400848410101010101010818181818181013A
:10C384000101010101010101010101010101010199
:10C394000101011010101010108282828282820228
:10C3A4000202020202020202020202020202020269
:10C3B40002020210101010200007032004170201CB
:10C3C400085710408000000030C3020034C402004B
:10C3D40048C5020053756E004D6F6E0054756500BC
:10C3E40057656400546875004672690053617400AF
:10C3F400000000004A616E00466562004D617200F3
:10C40400417072004D6179004A756E004A756C0086
:10C4140041756700536570004F6374004E6F76007A
:10C424004465630000000000414D00504D000000D1
:10C434006CC5020068C5020068C5020068C5020038
:10C4440068C5020068C5020068C5020068C502002C
:10C4540068C5020068C50200FFFFFFFFFFFFFFFF82
:10C46400FFFFFFFFFFFF0000A8C40200D8C30200C3
:10C47400E4C40200F8C302002CC402008CC402000D
:10C484003CC5020098C40200256D2F25642F257930
:10C494000000000025612025622025652025542008
:10C4A4002559000053756E646179004D6F6E6461A7
:10C4B400790054756573646179005765646E6573BA
:10C4C40064617900546875727364617900467269B5
:10C4D40064617900536174757264617900000000CD
:10C4E4004A616E756172790046656272756172792E
:10C4F400004D6172636800417072696C004D61792E
:10C50400004A756E65004A756C79004175677573EC
:10C51400740053657074656D626572004F63746F67
:10C52400626572004E6F76656D6265720044656384
:10C53400656D62657200000025483A254D3A255321
:10C5440000000000ADB30200C9B30200D5B302007D
:10C55400E1B30200FDB3020009B4020015B4020005
:0AC5640023B40200000000002E00C6
:10C5700000000000FF000000001001401100040056
:10C5800000000000002000400000000000200040EB
:10C59000000000000090D003010002001400FFFF23
:10C5A000000000000000000000000000000000008B
:10C5B00000000000242B0020000000006438002050
:10C5C00001000400CCC30200CCC30200CCC30200B3
:08C5D000CCC30200CCC3020041
:040000032000637501
:00000001FF
